:1000000001007370043073504030971100209381C9
:100010006182170200201302E21A17110020130157
:1000200061FE9302002073A0027D9302000873A07A
:10003000027D970200009382E20C7390523093028B
:10004000F00373B0523073E0513073F00232130595
:100050000011970500209385E5FA6300B5021706A5
:1000600000201306E6FC63FAC5008322050023A0E6
:10007000550011059105E3EAC5FE1725000013059B
:10008000E577970500209385E5FA6300B50217062A
:1000900000201306261363FAC5008322050023A05F
:1000A000550011059105E3EAC5FE1705002013056B
:1000B0006511971500209385E5B46377B50023207B
:1000C00005001105E36DB5FEEF005040EF00303A3A
:1000D00001458145EF20805AEF00F03D01A013005B
:1000E00000001300000013000000130000001300C4
:1000F00000001300000013000000130000000100C6
:1001000073005010F5BF0100130000001300000041
:10011000611106C222C02000B707002093870700A4
:10012000BE85896713850773972000E0E780E02E7E
:0C01300081473E859240024421018280FC
:1001800001A00000000000000000000000000000CE
:10019000000000000000000000000000000000005F
:1001A000000000000000000000000000000000004F
:1001B000000000000000000000000000000000003F
:1001C000130181FC06C012C216C41AC61EC82ACA70
:1001D0002ECC32CE36D03AD23ED473D0E57E735098
:1001E000F67E73D0B67E732520348A854929D25293
:1001F0007390427CC25273901234B2527390223484
:1002000082401242A2423243C2435245E245724604
:1002100082561257A2571301810373002030010048
:100220001300000013000000130000001300000082
:10023000130000001300000013000000130181FCF4
:1002400006C012C216C41AC61EC82ACA2ECC32CE86
:1002500036D03AD23ED473D0E57E7350F67E73D05A
:10026000B67EF390D07E73700430D2527390427C8D
:10027000C25273901234B2527390223482401242AE
:10028000A2423243C2435245E24572468256125759
:10029000A2571301810373002030130181F186D32B
:1002A000A2D1A011232AA4F2232CB4F2930784FF35
:1002B000232CF4F0832784F1938747F49D078D83E3
:1002C00013953700B70703182326F4F88327C4F8DB
:1002D00091072324F4F8832784F89C432322F4F81D
:1002E000832744F82324F4F68327C4F82320F4F862
:1002F000832704F89C43232EF4F68327C4F7232294
:10030000F4F68327C4F89107232CF4F6832784F7A7
:100310009C43232AF4F6832744F72320F4F603278B
:1003200084F6832704F6630FF7008327C4F8232895
:10033000F4F6832704F79C432326F4F68327C4F6B8
:100340002322F4F6832704F6232EF4F0232004F26C
:100350008327C4F1939607000146832744F63E8322
:100360008143B36766001CC1B3E776005CC11841E6
:100370005C4118CD5CCD032744F3832784F303232A
:1003800085018323C50133066700B285B3B5E50057
:10039000B3867700B387D500BE863287B68718C983
:1003A0005CC9232604FC18495C4918C55CC5832731
:1003B000C4FC2324F4FC832784FCB5E7B7070318A7
:1003C000A1072322F4FC832744FC2320F4FCFD57DF
:1003D000232EF4FA8327C4FB032704FC1CC301006B
:1003E000832744FC91075845135707002326E4F25E
:1003F000232804F20327C4F2232CF4FA232AE4FA74
:10040000832744FB032784FB1CC301001C450327EF
:1004100044FC2328E4FA2326F4FA8327C4FA0327AA
:1004200004FB1CC395A8832784FC13973700B75798
:100430000318BA972324F4FA832784FA2322F4FAC0
:10044000FD572320F4FA832704FA032744FA1CC338
:100450000100832784FA9107584513570700232288
:10046000E4F2232404F2032744F2232EF4F8232C8D
:10047000E4F8832784F90327C4F91CC301001C4551
:10048000032784FA232AE4F82328F4F8832704F9BD
:10049000032744F91CC30100010001009D47232AE2
:1004A000F4FC232804FC37070218832744FD9387B4
:1004B00007408A07BA9783C7270093F7F70FB70655
:1004C0000218F99B13F7F70F832744FD9387074022
:1004D0008A07B6972381E70037070218832744FD70
:1004E000938707408A07BA9783C7270013F7F70F48
:1004F000832704FD93F7F70FB7060218D98F13F778
:10050000F70F832744FD938707408A07B697238117
:10051000E70001009D472328F4FEA30704FEB70768
:10052000021883C7070093F7F70F8583BD8B230756
:10053000F4FE8D47A306F4FE8347E4FEF9C70347A4
:10054000E4FE8347D4FE63F6E7008347D4FE230727
:10055000F4FE8347E4FE0547B317F70093F7F70F60
:10056000FD172306F4FE0347F4FE8347C4FE63F63B
:10057000E7008347C4FEA307F4FE0347F4FE834766
:10058000E4FEA146B387F640B317F700A305F4FED7
:10059000832704FF2322F4FE37070218832744FE33
:1005A000938707408A07BA9783C7370093F7F70FF7
:1005B000A301F4FE034734FE8347E4FEB317F700BC
:1005C000A301F4FE034734FE8347E4FEB357F7402C
:1005D000A301F4FE8347B4FE3E87834734FED98FE0
:1005E00093F7F70F032704FF232EE4FCA30DF4FC7D
:1005F000370702188327C4FD938707408A07BA97F5
:100600000347B4FDA381E70011A001009D47232A01
:10061000F4FE37070218832744FF938707408A07B1
:10062000BA9783C7170093F7F70FB706021893E737
:10063000170013F7F70F832744FF938707408A07B4
:10064000B697A380E700010081473E859E500E5477
:100650001301810E8280311106C822C6400823286A
:10066000A4FE2326B4FE8547232AF4FE832744FFF5
:1006700073B007817300501001000100EDB7211124
:1006800006CA22C820082326A4FE2324B4FE03277A
:10069000C4FE8567FD17F98F232AF4FE232804FE84
:1006A000032744FF8567FD176302F702032744FF12
:1006B000AD4763EAE7001387C19A832744FF8A079F
:1006C000BA979C4331A09307606519A083A7C1998D
:1006D0002328F4FE832704FF81CB832704FF83258F
:1006E00084FE0325C4FE829781473E85D240424462
:1006F00061018280411106C622C4000813076065AB
:1007000023AEE198232A04FE39A813076065938677
:10071000C19A832744FF8A07B69798C3832744FF6B
:100720008507232AF4FE032744FFAD47E3DFE7FCF8
:100730009307001C93E737002328F4FE832704FF68
:10074000739057300100B240224441018280211150
:1007500006CA22C820089387018D232AF4FE832726
:1007600044FF739077309307C02393E71700232843
:10077000F4FE832704FF7390C77EA30504FEB7072A
:1007800002180347B4FEA385E70001008D47232626
:10079000F4FEB707021883C7070013F7F70FB70770
:1007A0000218059B1377F70F2380E700B70702189D
:1007B00083C7070093F7F70F139747608327C4FE9B
:1007C00093974760860793974760F98B93974760A5
:1007D000D98F13974760B70702181377F70F238055
:1007E000E70001000100D240424461018280130110
:1007F00041FA86CCA2CAE0082324A4FA2322B4FA40
:10080000032784FA9307100263E5E700832744FA7D
:1008100099E3FD5749A6832744FA83C7170093B786
:10082000170093F7F70F3E87832784FA2328F4FAFB
:100830002326E4FA37070218832704FB938707402F
:100840008A07BA9783C7270093F7F70FB7060218EE
:10085000F99B13F7F70F832704FB938707408A0759
:10086000B6972381E70037070218832704FB938795
:1008700007408A07BA9783C7270013F7F70F832724
:10088000C4FA93F7F70FB7060218D98F13F7F70FCB
:10089000832704FB938707408A07B6972381E700E5
:1008A0000100832744FA83C707003E87832784FA21
:1008B000232CF4FA232AE4FA37070218832784FB4F
:1008C000938707408A07BA9783C7270093F7F70FE4
:1008D000B7060218E59B13F7F70F832784FB93876E
:1008E00007408A07B6972381E70037070218832756
:1008F00084FB938707408A07BA9783C7270013F7BB
:10090000F70F832744FB93F7F70F860793F7F70F4B
:10091000B7060218D98F13F7F70F832784FB938745
:1009200007408A07B6972381E7000100832744FA2E
:1009300083C72700032784FA232AE4FCA309F4FCD5
:10094000B707021883C7070093F7F70F8583BD8B9E
:100950002309F4FC8D47A308F4FC834724FDF9C761
:10096000034724FD834714FD63F6E700834714FD26
:100970002309F4FC834724FD0547B317F70093F7D9
:10098000F70FFD172308F4FC034734FD834704FDEC
:1009900063F6E700834704FDA309F4FC034734FD35
:1009A000834724FDA146B387F640B317F700A3079A
:1009B000F4FC832744FD2324F4FC37070218832723
:1009C00084FC938707408A07BA9783C7370093F759
:1009D000F70FA303F4FC034774FC834724FDB3170C
:1009E000F700A303F4FC034774FC834724FDB357CB
:1009F000F740A303F4FC8347F4FC3E87834774FC71
:100A0000D98F93F7F70F032744FD2320E4FCA30FAE
:100A1000F4FA37070218832704FC938707408A07F4
:100A2000BA970347F4FBA381E70011A001008327D5
:100A300044FA83C73700032784FA2328E4FEA30778
:100A4000F4FEB707021883C7070093F7F70F8583F3
:100A5000BD8B2307F4FE8D47A306F4FE0347E4FE97
:100A60008347D4FE6378F70E0347D4FE8347E4FE42
:100A7000B307F7400547B317F70093F7F70FFD17D4
:100A80002306F4FE0347F4FE8347C4FE63F6E70043
:100A90008347C4FEA307F4FE0347F4FE8347D4FE56
:100AA000A146B387F640B317F700A307F4FE8347C8
:100AB000D4FE1307F00FB357F740A305F4FE8347A6
:100AC000F4FE3E878347B4FED98FA307F4FE832745
:100AD00004FF2322F4FE37070218832744FE93877E
:100AE00007408A07BA9783C7370093F7F70FA30128
:100AF000F4FE034734FE8347E4FEA146B387F64085
:100B0000B357F740A301F4FE034734FE8347E4FEE6
:100B1000A146B387F640B317F700A301F4FE83475D
:100B2000F4FE3E87834734FED98F93F7F70F0327F0
:100B300004FF232EE4FCA30DF4FC370702188327DF
:100B4000C4FD938707408A07BA970347B4FDA38182
:100B5000E70001000100832784FA232AF4FE370707
:100B60000218832744FF938707408A07BA9783C7F1
:100B7000170093F7F70FB706021893E7170013F75C
:100B8000F70F832744FF938707408A07B697A38010
:100B9000E700010081473E85E64056441301C10548
:100BA0008280130181FD06D222D020102320A4FED2
:100BB000232EB4FC232CC4FC032704FE930710024D
:100BC00063E8E7008327C4FD81C7832784FD99E399
:100BD000FD5741A8832704FE232AF4FE3707021895
:100BE000832744FF938707408A07BA9783C7170074
:100BF00093F7F70FB7060218F99B13F7F70F832740
:100C000044FF938707408A07B697A380E700010057
:100C10008327C4FDA9C38327C4FD032704FE23281B
:100C2000E4FE2326F4FEF32770302324F4FE83270A
:100C300084FE2322F4FE832704FF139727008327D3
:100C400044FEBA972322F4FE832744FE3E8783277F
:100C5000C4FE1CC30100832584FD032504FE413E20
:100C600081473E85925002541301810282806111B6
:100C700006C222C02000370703188567BA9783A7EA
:100C800087FFB706031813E717008567B69723ACED
:100C9000E7FE010023AA019823A801987D202A8756
:100CA000B707002023A8E702B13455340100924071
:100CB000024421018280511106C422C26000232A0D
:100CC000A4FE0100A240124431018280611106C2DB
:100CD00022C02000B7070140938707803707A5A5EA
:100CE0001307070298C3B7070140938707807D5712
:100CF000D8C3B7070140938707809C5713F707E0D5
:100D0000B7070140938707801367C71398D7B7F7D2
:100D100001409857B7F701401317F72898D7B767DE
:100D20000040938707809853C177B376F700B76781
:100D3000004093870780216713070708558F98D3D2
:100D400001009240024421018280511106C422C256
:100D50006000B7F701409C539D8B91EBB7070020D3
:100D6000378793031307077023A8E702ADA8B7F7E7
:100D700001409C5313F777008D476318F700B707BE
:100D80000020216723A8E702B9A8B7F701409C53C8
:100D900013F777008547631BF700B7070020371765
:100DA0007A001307072023A8E70235A8B7F7014008
:100DB0009C53A183BD8B232AF4FE832744FF89C75C
:100DC000832744FF850711A08947232AF4FEB787AC
:100DD000930313870770832744FF3357F702B7073E
:100DE000002023A8E702B707002083A707033E855A
:100DF000A240124431018280011106CE22CC0010A3
:100E00002320A4FE232204FEB78793039387077051
:100E1000232AF4FEB7F701409C5313F77700894764
:100E2000631DF702B7F701409C53A183BD8B2328B4
:100E3000F4FE832704FF89C7832704FF850711A0D9
:100E400089472328F4FEB787930313870770832706
:100E500004FFB357F702232AF4FEB7F701409C536F
:100E6000E1838D8B2322F4FE032744FE8547631C18
:100E7000F700032744FFB7576210938737DDB33776
:100E8000F7029D8389A0032744FE8947631CF7006E
:100E9000032744FFB7576210938737DDB337F70254
:100EA000A18315A0032744FE8D47631CF700032789
:100EB00044FFB7576210938737DDB337F702A58336
:100EC00019A09307000223ACF198032704FE85477D
:100ED0006319F70003A78199BA878A07BA9786072B
:100EE000A1A0032704FE8947631CF70003A781998B
:100EF000BA878A07BA9713972700BA978A072DA04F
:100F0000032704FE8D47631FF70003A78199BA8763
:100F10008A07BA9713972700BA9713972700BA97AB
:100F20008E0719A083A7819923AAF198A1472324AA
:100F3000F4FE832784FE73B00730010037070318DF
:100F40008567BA9783A787FFB705031813E71700CC
:100F50008567AE9723ACE7FE010083A741993E86E3
:100F600081463285B685EFF04FB3370703188567A2
:100F7000BA9783A787FFB706031813F7E7FF8567BC
:100F8000B69723ACE7FE0100A1472326F4FE832792
:100F9000C4FE73A0073001000100F2406244056105
:100FA0008280130141EA232C1114232A8114E00AC0
:100FB000930784FF2322F4EA832744EA938787EE8A
:100FC0009D078D831395370083A701991387170019
:100FD00023A8E19883A741993E86814630C174C118
:100FE000B7070318232AF4FE832744FF9107232819
:100FF000F4FE832704FF9C432326F4FE8327C4FECC
:10100000232AF4F2832744FF2324F4FE832784FE5B
:101010009C432322F4FE832744FE2328F4F28327F3
:1010200044FF91072320F4FE832704FE9C43232ED4
:10103000F4FC8327C4FD2326F4F2032744F383271B
:10104000C4F2630FF700832744FF232CF4FC8327AB
:1010500084FD9C43232AF4FC832744FD2328F4F2D7
:101060008327C4F2232CF4EC232E04EC832784ED95
:10107000939307000143832704F32328F4EC232AE6
:1010800004EC832604ED032744EDB687B367F30031
:101090001CDDBA87B3E7F3005CDD185D5C5D18D931
:1010A0005CD938417C41105954593303C7009A85A3
:1010B000B3B5E500B383D700B3877500BE8323249F
:1010C000650223267502854658555C5963EBE70097
:1010D00058555C596316F70018551C5963E3E7002F
:1010E000814693F7F60F6383071018555C5518D1A6
:1010F0005CD1232804FC18515C5118CD5CCD8327AA
:1011000004FD2326F4FC8327C4FCB5E7B7070318C6
:10111000A1072324F4FC832784FC2322F4FCFD573D
:101120002320F4FC832704FC032744FC1CC3010098
:10113000832784FC9107584D135707002324E4ECC0
:10114000232604EC032784EC232EF4FA232CE4FA60
:10115000832784FB0327C4FB1CC301001C4D03270A
:1011600084FC232AE4FA2328F4FA832704FB0327C8
:1011700044FB1CC395A88327C4FC13973700B757BB
:101180000318BA972326F4FA8327C4FA2324F4FA1F
:10119000FD572322F4FA832744FA032784FA1CC359
:1011A00001008327C4FA9107584D135707002320E5
:1011B000E4EC232204EC032704EC2320F4FA232E8E
:1011C000E4F88327C4F9032704FA1CC301001C4D6B
:1011D0000327C4FA232CE4F8232AF4F8832744F9DC
:1011E000032784F91CC30100010095AA0147814728
:1011F00018C95CC9B70703182328F4F8832704F932
:101200002326F4F8232404F8832784F80327C4F85A
:101210001CC30100832704F991075849135707009D
:10122000232CE4EA232E04EA032784EB2322F4F898
:101230002320E4F8832704F8032744F81CC30100A3
:101240001C49032704F9232EE4F6232CF4F6832704
:1012500084F70327C4F71CC30100010038417C4117
:1012600018C55CC5232A04F618455C4518C15CC145
:10127000832744F72328F4F6832704F7B5E7B70755
:101280000318A1072326F4F68327C4F62324F4F6D3
:10129000FD572322F4F6832744F6032784F61CC364
:1012A00001008327C4F691075841135707002328EC
:1012B000E4EA232A04EA032704EB2320F4F6232E8E
:1012C000E4F48327C4F5032704F61CC301001C4182
:1012D0000327C4F6232CE4F4232AF4F4832744F5EB
:1012E000032784F51CC395A8832704F713973700B9
:1012F000B7570318BA972328F4F4832704F5232655
:10130000F4F4FD572324F4F4832784F40327C4F46E
:101310001CC30100832704F59107584113570700A8
:101320002324E4EA232604EA032784EA2322F4F4AC
:101330002320E4F4832704F4032744F41CC30100AE
:101340001C41032704F5232EE4F2232CF4F2832717
:1013500084F30327C4F31CC3010001000100010052
:1013600083208115032441151301C11582801301C7
:1013700041FA86CCA2CAB6C8BAC6BEC4E008F327F2
:1013800020342324F4FE832784FE2322F4FEF32753
:1013900010342320F4FE832704FE232EF4FCF327CD
:1013A000407C232CF4FC832784FD232AF4FCA147F2
:1013B0002322F4FA832744FA73A007300100232C78
:1013C00004FA832784FB232AF4FA832744FB85E36A
:1013D000370703188567BA9783A7C7FFB7060318AF
:1013E00013F7E7FF8567B69723AEE7FE35A083279F
:1013F00044FB13972700B7170318BA972328F4FA6A
:10140000832704FB2326F4FA232404FA832784FA8F
:101410000327C4FA1CC301000100010001008D472D
:101420002320F4FC832704FC232EF4FA3707021848
:101430008327C4FB938707408A07BA9783C70700AF
:1014400093F7F70FB7060218F99B13F7F70F8327E7
:10145000C4FB938707408A07B6972380E700010003
:101460000100A1472322F4FC832744FC73B007301A
:101470000100832744FD2328F4FC832704FD739097
:10148000477C8327C4FD2326F4FC8327C4FC739088
:101490001734832744FE2324F4FC832784FC7390B1
:1014A00027340100E6405644C6463647A647130196
:1014B000C10573002030611106C222C02000010066
:1014C00092400244210173002030611106C222C003
:1014D000200001009240024421017300203041119C
:1014E00006C622C400082328A4FEB7F7014098537B
:1014F000FD779387870FB376F700832704FF984320
:10150000832704FFDC435D8F8567938777F07D8FAA
:10151000B7F70140558F98D3832704FF9C47232AB0
:10152000F4FEB7F701409853B70700FDFD17B376F7
:10153000F700032744FFB70700037D8FB7F701408B
:10154000558F98D30100EFF05F802A87B7070020FE
:1015500023A8E7020100B240224441018280011128
:1015600006CE22CC00102322A4FE2320B4FEB7070F
:10157000002083A70703232AF4FE232804FE8327E1
:1015800044FE81C7832704FE99E38547E1A803272A
:1015900044FEB72700406319F702B7F70140985798
:1015A000B7F701401367170098D7B7F70140D85332
:1015B000B7F7014013671700D8D3B7F70140D853E6
:1015C000B7F70140799BD8D3832744FE23A20700B5
:1015D000832744FE23A60700832744FE2324F4FE2A
:1015E000832784FE3D671307079398D30100832761
:1015F00044FE2326F4FE8327C4FE3D6713070793AA
:10160000D8CF0100832704FE9C431397370083271C
:1016100044FF3E97832704FE9C439207B357F7028B
:101620002328F4FE832744FE032704FF98C783275B
:1016300044FEDC4313F707EC832704FED4438327DF
:1016400004FE9C47DD8E832704FEDC47DD8E832766
:1016500004FE9C4BD58F93F7F7135D8F832744FED1
:10166000D8C381473E85F2406244056182804111C2
:1016700006C622C40008232AA4FEAE872319F4FE5E
:10168000835724FF93F7F71F33C70708832744FFC7
:101690001377F71F944393F606E0558F98C3010024
:1016A000B240224441018280511106C422C260002E
:1016B000232AA4FE832744FF9C4393F7F71FB3C755
:1016C00007083E85A240124431018280311106C8CC
:1016D00022C64008232AA4FE2328B4FE2326C4FEE3
:1016E000832744FF99E3854715A88327C4FE99CB38
:1016F000832744FFD847832704FF5D8F832744FF58
:10170000D8C721A8832744FFD847832704FF93C75E
:10171000F7FF7D8F832744FFD8C781473E85C240AE
:10172000324451018280130141FD06D422D260105F
:10173000232CA4FC232AB4FC232804FE032784FDC5
:10174000B7170140631BF700B7F70140F843B7F73D
:10175000014013671700F8C339A8032784FDB72792
:101760000140631AF700B7F70140F843B7F70140AB
:1017700013672700F8C3232A04FE99A6832744FF92
:101780000547B317F7002326F4FE832744FD83D7CC
:1017900007003E878327C4FEF98F638B07308327BA
:1017A00084FDF84F8327C4FE5D8F832784FDF8CF27
:1017B000832744FDD8478547631CF700832784FDB2
:1017C000F8438327C4FE5D8F832784FDF8C311A8E7
:1017D000832784FDB8478327C4FE5D8F832784FD5C
:1017E000B8C7832744FDDC4311476388E7161147D8
:1017F000636EF7000D476385E7180D476368F700D0
:1018000005476385E70C09476386E712832784FD54
:10181000D84B8327C4FE5D8F832784FDD8CB8327D5
:1018200084FD984F8327C4FE5D8F832784FD98CF66
:10183000832744FD984785476315F702832784FD76
:10184000D85F8327C4FE5D8F832784FDD8DF83277D
:1018500084FDB84B8327C4FE5D8F832784FDB8CBFE
:10186000A1A8832744FD984789476315F70283277A
:1018700084FDF8478327C4FE5D8F832784FDF8C766
:10188000832784FDB8438327C4FE5D8F832784FDAF
:10189000B8C31DA0832784FDB84B8327C4FE5D8F8A
:1018A000832784FDB8CB832784FDB8438327C4FEF8
:1018B0005D8F832784FDB8C3832744FDD1073E860F
:1018C0008325C4FE032584FD092CF5A2832784FD0E
:1018D000D84F8327C4FE5D8F832784FDD8CF83270D
:1018E00084FD984B8327C4FE5D8F832784FD98CBAE
:1018F000832744FD98478547631CF700832784FDB1
:10190000D8438327C4FE5D8F832784FDD8C35DA29F
:10191000832744FD98478947631EF718832784FD72
:10192000D8438327C4FE93C7F7FF7D8F832784FDA9
:10193000D8C349A2832784FDD84F8327C4FE5D8F77
:10194000832784FDD8CF832784FDB8538327C4FE23
:101950005D8F832784FDB8D3B9AA832784FDD84F30
:101960008327C4FE5D8F832784FDD8CF832784FD22
:10197000D84B8327C4FE5D8F832784FDD8CB25AA4F
:10198000032784FDB7170140631EF7080327C4FE31
:10199000B1679387F703F98FD1C78327C4FE23204C
:1019A000F4FE832704FE939707607D47B307F74053
:1019B0002324F4FE032784FE954763D6E70083279C
:1019C00084FEE11719A0832784FE2324F4FEB717B1
:1019D0000140938707079443032784FEBA8786074D
:1019E000BA971D47B317F70093C7F7FFFD8E8327FC
:1019F00044FD904B032784FEBA878607BA973316B7
:101A0000F600032784FEBA878607BA971D47B317E7
:101A1000F7003377F600B717014093870707558F14
:101A200098C371A0032784FDB7270140631FF70601
:101A30008327C4FE93F7F703ADCB8327C4FE232E81
:101A4000F4FC8327C4FD939707607D47B307F740F5
:101A50002322F4FEB717014093870707D4430327D7
:101A600044FEBA878607BA971D47B317F70093C796
:101A7000F7FFFD8E832744FD904B032744FEBA8772
:101A80008607BA973316F600032744FEBA878607FF
:101A9000BA971D47B317F7003377F600B717014021
:101AA00093870707558FD8C319A0FD570DA021A014
:101AB000010011A00100832744FF8507232AF4FEBB
:101AC000032744FFBD47E3DBE7CA832704FF3E85C6
:101AD000A25012541301C1028280311106C822C6DD
:101AE0004008232AA4FE2328B4FE2326C4FE83270D
:101AF000C4FED8438947631CF700832744FF9847F7
:101B0000832704FF5D8F832744FF98C7A1A88327FD
:101B1000C4FED84385476315F702832744FFD8479F
:101B2000832704FF5D8F832744FFD8C7832744FFA3
:101B30009857832704FF5D8F832744FF98D71DA004
:101B4000832744FFD847832704FF5D8F832744FF03
:101B5000D8C7832744FFD857832704FF5D8F832787
:101B600044FFD8D78327C4FE98438547631CF700FA
:101B7000832744FF985B832704FF5D8F832744FFFF
:101B800098DB19A8832744FFD85B832704FF5D8F68
:101B9000832744FFD8DB0100C240324451018280D8
:101BA000828019C16F0080788280AA95AA8703C7B6
:101BB000070019C36395B7003385A7408280850766
:101BC000FDB7130505FD1335A500828062B8AA8410
:101BD00001449C4003C507003EC0E53782472947C2
:101BE00019E1228562BE3304E4029386170094C093
:101BF00083C70700938707FD3E94E1BF6AB83AC4E4
:101C000052572EC036C20D8B2A84B28431CBB28299
:101C10003E87338557003306E54029E7D257898B45
:101C200081CBB307954042573385F40063ECE7045A
:101C30006ABE924682453EC83AC613050002029427
:101C40003247C2470507C2563386F4403A96E362EC
:101C5000D7FE814263E4F600B382F640A6924DBF00
:101C60003E87D5B73ECAA2477D1792463385E70027
:101C700082450345050016C83AC60294D247C242BF
:101C8000324741BF924682453EC42A861305000270
:101C90000294A247850741BF66B832C442562AC0A3
:101CA0002EC293732600034301021255A252B2556D
:101CB000639403049373160089C963880300631552
:101CC00003001374C60011C0FD159304000331A076
:101CD0003304F70023009400850763F5570013B41D
:101CE00007027DF4638A03001304000363F6B70060
:101CF00093B3070263970308937306016380030697
:101D0000937306406391030299CF63845700639CE9
:101D1000B7009382F7FF63870200930305FFF9176B
:101D2000638603009687C142631A550693720602C2
:101D3000FD43639E020463E3F3063305F700930259
:101D400080072300550085077D456365F50233054F
:101D5000F700930200032300550085077D45636B60
:101D6000F500630703043305F7001303D0022300D3
:101D70006500850732D22ED022469245024566BACA
:101D8000B5BDB303F70023808300850785B763E7FC
:101D9000F3003305F7009302800565B779154DF51B
:101DA00013B5070255D13305F7009302200651BF42
:101DB0001375460011C53305F7001303B00245BF84
:101DC0001375860045D93305F7001303000245B7A4
:101DD0006EB861113ECC36CAA647564325EB137444
:101DE000F3FE137303406315030413535448930223
:101DF00010066304030093021004BA8364080147C9
:101E0000D91233F3F302A5461373F30F63E46604A8
:101E1000130303031373F30F23806400050733D305
:101E2000F302850463E6F300930307FE6392030263
:101E300046433EC2E2471AC63643D2463EC022C897
:101E40001AC4BA877808893D21016EBE1A8471BF11
:101E50009A8345BF16937DBF6EB841112ACA2ECC16
:101E600032C8B6C089E58967938707BA3ECA01437D
:101E7000864703C507000DE1C2471A866364F30075
:101E80001386F7FFC246E245D2471ACE0145829734
:101E9000724341011A856EBE9386170036D29306AF
:101EA0005002630DD500C246E245D2473ACE1A86AB
:101EB0001304130082977247228389AC938617001C
:101EC000B6C08907014601449306B0029303D002CD
:101ED00093020003930500021305300283C4F7FF49
:101EE000638ED40E63E0960E638DB40E638EA40EE3
:101EF000FD1711C2BEC026853AD23ED01ACED131CE
:101F000072438257125765C588003AD01ACE7D3980
:101F100072430257AA8286449306E002814703C6B1
:101F20000400631FD60293861400B6C083C6140053
:101F30003AD61AD436853ED216D036CE5931F2462C
:101F400082522253325713640440814761C588008E
:101F50003AD21AD016CE9D39F24202531257AA87AE
:101F600006461305C00683450600930616006385E2
:101F7000A50C636CB50A13058006638DA50C1305CB
:101F8000A0066384A50EB28603C50600850636D278
:101F900093058007E3E9A5F09306300663EAA60CF3
:101FA000130620066307C516630ED51A9306500262
:101FB000E30BD5EE93068005E317D5EE1364040218
:101FC000C146D5A863897400E39454F213641400E5
:101FD0008507054621B713642400DDBF1364440060
:101FE000C5BF13648400EDB713640401D5B793062D
:101FF000A0028142E391D4F28322070093064700B6
:1020000063D6020013642400B30250408507BEC0AB
:10201000368711B71306A002E394C6F41C43890463
:10202000A6C0B3E7070A110725BF1305A007E39C65
:10203000A5F41364041029A803451600B6C063056F
:10204000B5001364041089B71364043093062600A6
:10205000B6C01DBF03451600B6C06305B5001364C6
:1020600004081DB71364040CD5B713640420CDB75E
:10207000371612009306C5F913061682B353D648D5
:102080006396030293063007630FD5169306000785
:10209000E31BD5E093044700136414021843A146E0
:1020A0003EC2C14722C636C43EC071A81306F00620
:1020B000A1466312C524130675F909C61306C5F9AE
:1020C00011C24D981376044011C27998930575F9A1
:1020D0001376042081C51305C5F939E905EA13769D
:1020E00004109304470005CA18433306E0403EC27B
:1020F00022C69357F70116C436C03367C70AC246D3
:10210000E24552451A86E9312A8326879257BEC096
:1021100085B389464DB713760404184301C6137777
:10212000F70FE1B71376040869D21317576075BF2C
:1021300071FE137604109304470001CA184322C6A7
:1021400016C43EC236C081475DBF137604041843EF
:1021500001C61377F70FE5B7137604086DD233473E
:102160000708F1BF0988854721E0814429A8C246B4
:10217000E245D2473AD41AD016CE13050002829710
:10218000F24202532257330693008504E3E154FEE2
:1021900033365000894763840200938712008146DA
:1021A00019C29386F2FF36933ED4930747003ECE82
:1021B000C246D247E2450345070016D01A8693046B
:1021C000130082978252A25705CC3E8426860DA02A
:1021D0003ED6C246D247E2451307160016D43AD07F
:1021E0001305000282970257A252B25705043A869D
:1021F000E36054FE014763E4F2003387F240BA948F
:102200007247268321B793064700184336D6FD55FB
:102210003AD091C3BE8502551ADA3ED816CE713235
:10222000937704403ED43E87F242C2575253AA8469
:1022300019C3B354F50A137724003ACE1DEF1A865A
:1022400005A03EDAC246D247E2451ADC16D813058D
:102250000002130416008297C252D257625322869C
:10226000338764403297E36E57FC014763E4920082
:10227000338792408504BA943A931A8415A0BA879A
:102280003EDCC246D247E245130714001ADE16DAD6
:102290003AD8228682974257D252E25772533A84F2
:1022A00082563307644036970345070011C522570D
:1022B00061DB1387F7FFE1F7F2479DCB228631A858
:1022C000930716003ECEC246D247E24516D013050C
:1022D00000028297F24782523E86B3878440B297CB
:1022E000E3E057FE814763E49200B38792403E9457
:1022F0003257228321BD6375A600C146E30DB5DACE
:102300003D98A9464DBB011136CAAA8609652EC65D
:1023100032C83ACC8A8578007D56130525BA06C4A2
:102320003ECE3AC2153EA24005618280411106C6EA
:1023300022C40008AA87A309F4FE834734FFB3C769
:102340000708BE8537250040EFF06FB2B727004081
:10235000232AF4FE0100832744FF9C4B898BE5DF91
:1023600001000100B2402244410182801301C1F901
:1023700086D096CE9ACC9ECAA2C8AAC6AEC4B2C215
:10238000B6C03ADE3EDCC010F32720342328F4FC2C
:10239000832704FD2326F4FCF32710342324F4FCC4
:1023A000832784FC2322F4FCF327407C2320F4FCC5
:1023B000832704FC232EF4FAA1472324F4FA83276D
:1023C00084FA73A007300100ADA837250040EFF074
:1023D000AFADAA87A307F4FA83A7819AB5E303A751
:1023E000019A9307E00363EAE70483A7019A9386BF
:1023F000170023A0D19A1387C19DBA970347F4FA17
:102400002380E7000347F4FAB5476307F700034763
:10241000F4FAA9476317F70283A7019A1387C19DAE
:10242000BA972380070003A7019A23A2E19A23A069
:10243000019A054723A4E19A29A023A0019A11A09B
:102440000100B72700402322F4FA85472320F4FA3D
:10245000832744FA984B832704FAF98FBDF7A147E5
:10246000232EF4F88327C4F973B0073001008327C3
:10247000C4FB232CF4FA832784FB7390477C8327C7
:1024800044FC232AF4FA832744FB739017348327F0
:10249000C4FC2328F4FA832704FB7390273401003B
:1024A0008650F6426643D64346443645A645164610
:1024B00086467257E25713014106730020302111FE
:1024C00006CA22C820082326A4FE2324B4FE83279C
:1024D000C4FE99C7832784FE81C783A7819A99E3A5
:1024E0008147ADA8832784FE1387F7FF83A7419A0E
:1024F00063E6E700832784FEFD1719A083A7419AAE
:102500002328F4FE232A04FE35A00327C4FE8327D4
:1025100044FFBA979386C19D032744FF369703472C
:1025200007001377F70F2380E700832744FF850711
:10253000232AF4FE032744FF832704FFE367F7FC05
:102540000327C4FE832704FFBA972380070023A232
:10255000019A23A4019A23A0019A85473E85D2407F
:10256000424461018280611106C222C0200083A71B
:10257000819A3E8592400244210182801301C1FB71
:1025800086C022DEC000232A04FC232C04FC232E58
:1025900004FC232004FE232204FE232404FE23261D
:1025A00004FE232004FC232204FC232404FC232611
:1025B00004FC232804FC232E04FAA147231AF4FC6C
:1025C00085472322F4FE8D47232CF4FC930744FD1A
:1025D000BE8537250140EFF00F9593070002231ABF
:1025E000F4FC85472322F4FE930744FDBE8537257E
:1025F0000140EFF04F93F167938707202320F4FC0D
:1026000085472322F4FCA1472324F4FC232604FC61
:10261000930700102328F4FC930704FCBE8537259C
:102620000040EFE0DFF30546854537250040EFF039
:10263000EF899307C4FB3E8689679385C736654556
:10264000EFE02FD6A1472328F4FE832704FF73A0D1
:10265000073001000100B7270040232AF4FE83273A
:1026600044FFDC4313E70708832744FFD8C3010076
:10267000010086407254130141048280130141FA23
:1026800086CCA2CAE008232204FE232404FE2326CB
:1026900004FE232204FE930744FE3E85EFE03FE460
:1026A0000145EFE06FF5D93D896713858775A1393D
:1026B000970700002328F4FE832704FFBE8589675F
:1026C0001385C777893189671385C7792D3989675C
:1026D0001385477B0D3997E0FF1FE780A092232ADF
:1026E00004FE03A70199832744FF1D8F9307803EB3
:1026F00063FAE70283A70199232AF4FEAD35AA877E
:1027000091CF930744FA930500043E854D3B930710
:1027100044FABE8589671385C77CF53689671385BA
:10272000477DD536010001006DBF000000000000AC
:102730001B5B33366D72756E206174206661737435
:1027400020617265613A202470633D20782530381D
:10275000580A1B5B6D0000001B5B33336D546869C6
:10276000732069732061206170702064656D6F2033
:1027700070726F6A6563740A1B5B6D006C6F672013
:102780006465627567206D6573736167653A2024BF
:1027900070633D2078253038580A00001B5B3332C7
:1027A0006D636F6C6F7220677265656E0A1B5B6D7F
:1027B000000000001B5B33336D636F6C6F72207918
:1027C000656C6C6F770A1B5B6D00000052583A20F5
:1027D00025730A001B5B33336D7777776868682C45
:1027E00020636F6C6F722079656C6C6F770A1B5B6E
:0427F0006D00000078
:1027F80000879303000000000000000000000000B4
:1028080000000000000000000000000000000000C0
:1028180000000000000000000000000000000000B0
:1028280000000000000000000000000000000000A0
:102838000000000000000000000000000000000090
:102848000000000000000000000000000000000080
:102858000000000000000000000000000000000070
:102868000000000000000000000000000000000060
:102878000000000000000000000000000000000050
:102888000000000000000000000000000000000040
:102898000000000000000000000000000000000030
:1028A8000000000000000000000000000000000020
:1028B8000000000000000000000000000000000010
:1028C8000000000080010000800100006E1300007D
:1028D800800100008001000080010000A20F0000BC
:1028E80080010000800100008001000080010000DC
:1028F80080010000800100008001000080010000CC
:1029080080010000B6140000CA1400008001000015
:1029180080010000800100008001000080010000AB
:10292800800100008001000080010000800100009B
:10293800800100008001000080010000800100008B
:10294800800100008001000000000000000000007D
:10295800000000000000000000000000000000006F
:10296800000000000000000000000000000000005F
:10297800000000000000000000000000000000004F
:00000001FF
